:1000000012C02AC041C028C027C026C026C024C0B4
:1000100023C022C021C020C01FC01EC01DC01CC0E4
:100020001BC01AC019C011241FBECFEDCDBF10E0F8
:10003000A0E6B0E0E2E5F2E003C0C89531960D928B
:10004000A036B107D1F710E0A0E6B0E001C01D92E4
:10005000A836B107E1F758C0D3CF1F920F920FB661
:100060000F9211248F939F9380916200909163006F
:10007000019690936300809362009F918F910F90FF
:100080000FBE0F901F9018951F920F920FB60F92F0
:1000900011242F933F938F939F9322B780916200F7
:1000A00090916300982F8827820F911D9093610093
:1000B0008093600020916000309161008091640025
:1000C000909165002817390740F480916000909165
:1000D0006100909365008093640012BE10926300EB
:1000E0001092620080916600909167000196909353
:1000F0006700809366009F918F913F912F910F90A1
:100100000FBE0F901F901895BB9A89B7826089BF68
:1001100085B7846085BF8BB780688BBF83B78160EC
:1001200083BF789483996AC0C39A10926700109233
:10013000660012BE10926300109262008FEF9FEF74
:1001400090936500809364008091660090916700B1
:100150000997C0F542B72091620030916300E091A9
:100160006400F0916500F695E795F695E795809126
:10017000640090916500322F2227240F311D8E0FCD
:100180009F1F2817390700F3809166009091670040
:10019000019690936700809366008E2F9F2F60E0FA
:1001A00071E02ED082BF8E2F9F2F892F990F990B30
:1001B0009093630080936200809166009091670045
:1001C000099740F2839BFECF62E070E082B72091F6
:1001D0006200309163004091640050916500322FBD
:1001E0002227280F311D4217530710F08399EECFB5
:1001F0006150704077FFEACF839B96CFC39892CF30
:1002000097FB092E07260AD077FD04D00CD006D024
:1002100000201AF4709561957F4F0895F6F7909538
:1002200081959F4F0895AA1BBB1B51E107C0AA1FD0
:10023000BB1FA617B70710F0A61BB70B881F991F87
:100240005A95A9F780959095682F792F8A2F9B2F23
:0202500008950F
:00000001FF
